:100000000829A0007F39201B803C0920A01B003C50
:1000100008008A01820700340334063409340C34A2
:1000200010341334163419341C341F34223425345C
:1000300028342B342E3431343334363439343C3490
:100040003F3441344434473449344C344E345134D1
:100050005334553458345A345C345E34603462342A
:100060006434663468346A346B346D346F3470349D
:1000700071347334743475347634783479347A3432
:100080007A347B347C347D347D347E347E347E34EB
:100090007F347F347F347F349620B4000408B60068
:1000A0000800A4002508A402031CA5032708A60233
:1000B000031CA7033709A2003509A300A20A0319EC
:1000C000A30A4130A900AC01AD01AE01AF01A80106
:1000D0003608840034099320841304212408AC07D3
:1000E0000318AD0A2508AD072608AE070318AF0AA6
:1000F0002708AF072D080120803EA1002F0801200E
:10010000803EA107210CA80700083404031C340614
:100110008000290303194130A9000319A20A031919
:10012000A30F6D280329841780050329A800053033
:10013000A8190530840000308A0028080739820792
:100140000134023404340834103420344034803410
:100150000F39A00083161F088F3930389F00831293
:100160000310A00DA00D1F08C139200401389F0005
:100170000030A1003230D2209F149F18BD281E08E5
:10018000A10083161E080329A301A200FF30A207C5
:10019000031CA307031C03290330A100E630D2206F
:1001A000C628A101FC3EA000A109031CDD28FF30E8
:1001B0000000A0070318D828A0076400A10FD728C3
:1001C0000800A2000230EC28A2000130EC28A200B6
:1001D0000630EC28A2000530A80023082102031DE8
:1001E000F3282208200204300318013003190230DA
:1001F0002805031DFF3003290038031DFF300405C7
:10020000031DFF30032983130313831264000800C6
:1002100089309F00BC01BD010230A820B800210830
:10022000B900BA01BB013808A0003908A100A30138
:100230002530E420BE003C08A0003D08A100A30139
:100240000030E120C0003E0884004008FC20C000CF
:10025000C10064004008410403192F29A92338086C
:10026000A0003908A100A3012530E420BE003C080D
:10027000A0003D08A100A3010130E120C0003E081C
:1002800084004008FC20C000C10064004008410414
:1002900003194B294E210A30C4200C293808A0002C
:1002A0003908A1000330A3009230E420BE003808D2
:1002B000A0003908A1000330A300FF30E720C000F0
:1002C0003E0884004008FC20C000C10064004008D3
:1002D00041040319782900304C207830B700B5016B
:1002E0008430A6000330A7000230A500BC305120A6
:1002F0003808A0003908A1000330A3004930E420E9
:10030000BE003808A0003908A1000330A3009230D5
:10031000E720C0003E0884004008FC20C000C10067
:100320006400400841040319A22900304C207830B1
:10033000B700B5014C30A6000430A7000230A5007C
:10034000BC3051203808A0003908A1000230A300B9
:10035000FF30E420BE003808A0003908A1000330B7
:10036000A3004930E720C0003E0884004008FC207C
:10037000C000C1006400400841040319CC290030CA
:100380004C207830B700B5014C30A6000430A700EF
:100390000330A500843051203808A0003908A1009E
:1003A0000230A300B630E420BE003808A0003908AF
:1003B000A1000230A300FF30E720C0003E08840007
:1003C0004008FC20C000C10064004008410403193B
:1003D000F62900304C207830B700B5011430A60063
:1003E0000530A7000230A500BC3051203808A0001D
:1003F0003908A1000230A3006D30E420BE003808A7
:10040000A0003908A1000230A300B630E720C000E8
:100410003E0884004008FC20C000C1006400400881
:1004200041040319202A00304C207830B700B50170
:100430001430A6000530A7000330A50084305120F9
:100440003808A0003908A1000230A3002530E420BC
:10045000BE003808A0003908A1000230A3006D30AA
:10046000E720C0003E0884004008FC20C000C10016
:1004700064004008410403194A2A00304C207830B7
:10048000B700B5011430A6000530A7000430A50060
:100490004C3051203808A0003908A1000130A300D9
:1004A000DB30E420BE003808A0003908A10002308B
:1004B000A3002530E720C0003E0884004008FC204F
:1004C000C000C1006400400841040319742A0030D0
:1004D0004C207830B700B501DC30A6000530A7000D
:1004E0000230A500BC3051203808A0003908A10016
:1004F0000130A3009130E420BE003808A000390884
:10050000A1000130A300DB30E720C0003E088400DA
:100510004008FC20C000C1006400400841040319E9
:100520009E2A00304C207830B700B501DC30A600A0
:100530000530A7000330A500843051203808A00002
:100540003908A1000130A3004930E420BE0038087A
:10055000A0003908A1000130A3009130E720C000BD
:100560003E0884004008FC20C000C1006400400830
:1005700041040319C82A00304C207830B700B50177
:10058000DC30A6000530A7000430A5004C30512017
:100590003808A0003908A1000130A3000030E42091
:1005A000BE003808A0003908A1000130A30049307E
:1005B000E720C0003E0884004008FC20C000C100C5
:1005C0006400400841040319F22A00304C207830BE
:1005D000B700B501A430A6000630A7000430A5007E
:1005E0004C3051203808A0003908A100A301B630D2
:1005F000E420BE003808A0003908A1000130A300A3
:100600000030E720C0003E0884004008FC20C00005
:10061000C10064004008410403191B2B00304C202A
:100620007830B700B501DC30A6000530A7000530F2
:10063000A500143051203808A0003908A100A301FA
:100640006E30E420BE003808A0003908A100A301E4
:10065000B630E720C0003E0884004008FC20C000FF
:10066000C1006400400841040319432B00304C20B2
:100670007830B700B501A430A6000630A7000530D9
:10068000A500DC3051203808A0003908A100A301E2
:100690002530E420BE003808A0003908A100A301DD
:1006A0006E30E720C0003E0884004008FC20C000F7
:1006B000C10064004008410403196A2B00304C203B
:1006C000E830B7000330B5000A30A700A500283095
:1006D000A60051200230A820B8002108B9000A3035
:1006E000C420BA0A0319BB0A3A08A0003B08A100BB
:1006F000A301C830E420BE003808A0003908A100DA
:10070000A3012530E420C0003E0884004008FC20FE
:10071000C000C1003808A0003908A100A3016E3054
:10072000E720C2004008410484004208FC20C200C7
:10073000C30064004208430403199F2BDD253808D9
:10074000A0003908A100A3012530E420031D6A2B75
:1007500008003808A0003908A1000330A300923037
:10076000E420BE003808A0003908A1000330A3002F
:10077000FF30E720C0003E0884004008FC20C00095
:10078000C1006400400841040319D32B00304C2001
:100790007830B700B501B930A6000430A7000230A8
:1007A000A500B93051203808A0003908A100033055
:1007B000A3004930E420BE003808A0003908A10099
:1007C0000330A3009230E720C0003E0884004008B8
:1007D000FC20C000C1006400400841040319FD2B47
:1007E00000304C207830B700B5013830A600053015
:1007F000A7000230A500B93051203808A000390800
:10080000A1000230A300FF30E420BE003808A000A1
:100810003908A1000330A3004930E720C0003E089A
:1008200084004008FC20C000C1006400400841046E
:100830000319272C00304C207830B700B501C530A3
:10084000A6000530A7000230A500B93051203808B5
:10085000A0003908A1000230A300B630E420BE0099
:100860003808A0003908A1000230A300FF30E720BB
:10087000C0003E0884004008FC20C000C1006400A5
:10088000400841040319512C00304C207830B70047
:10089000B501B930A6000430A7000330A50002302E
:1008A00051203808A0003908A1000230A3006D30A3
:1008B000E420BE003808A0003908A1000230A300DF
:1008C000B630E720C0003E0884004008FC20C0008D
:1008D000C10064004008410403197B2C00304C2007
:1008E0007830B700B5013830A6000530A7000330D6
:1008F000A500023051203808A0003908A1000230BC
:10090000A3002530E420BE003808A0003908A1006B
:100910000230A3006D30E720C0003E08840040088C
:10092000FC20C000C1006400400841040319A52C4C
:1009300000304C207830B700B501C530A600053036
:10094000A7000330A500023051203808A000390864
:10095000A1000130A300DB30E420BE003808A00075
:100960003908A1000230A3002530E720C0003E086E
:1009700084004008FC20C000C1006400400841041D
:100980000319CF2C00304C207830B700B501B930B6
:10099000A6000430A7000330A500543051203808C9
:1009A000A0003908A1000130A3009130E420BE006E
:1009B0003808A0003908A1000130A300DB30E7208F
:1009C000C0003E0884004008FC20C000C100640054
:1009D000400841040319F92C00304C207830B7004E
:1009E000B5013830A6000530A7000330A50054300B
:1009F00051203808A0003908A1000130A300493077
:100A0000E420BE003808A0003908A1000130A3008E
:100A10009130E720C0003E0884004008FC20C00060
:100A2000C1006400400841040319232D00304C200C
:100A30007830B700B501C530A6000530A7000330F7
:100A4000A500543051203808A0003908A100013019
:100A5000A3000030E420BE003808A0003908A1003F
:100A60000130A3004930E720C0003E088400400860
:100A7000FC20C000C10064004008410403194D2D52
:100A800000304C207830B700B501B930A6000430F2
:100A9000A7000330A500AD3051203808A000390868
:100AA000A100A301B630E420BE003808A000390838
:100AB000A1000130A3000030E720C0003E08840000
:100AC0004008FC20C000C100640040084104031934
:100AD000762D00304C207830B700B5013830A600B4
:100AE0000530A7000330A500AD3051203808A00024
:100AF0003908A100A3016E30E420BE003808A00030
:100B00003908A100A301B630E720C0003E088400E8
:100B10004008FC20C000C1006400400841040319E3
:100B20009E2D00304C207830B700B501C530A600AE
:100B30000530A7000330A500AD3051200230A820B9
:100B4000B8002108B900BA0A0319BB0A3A08A00084
:100B50003B08A100A301C830E420BE003808A00073
:100B60003908A100A3012530E420C0003E0884001C
:100B70004008FC20C000C1003808A0003908A100CE
:100B8000A3016E30E720C2004008410484004208FF
:100B9000FC20C200C3006400420843040319D12DA5
:100BA000DD250A30C4203808A0003908A100A301BF
:100BB0002530E420031D9E2D08003C08A0003D08C0
:100BC000A100A3010130EA20031D022EBC01BD01DA
:100BD000BA01BB0100304C204B30B700B5010630E4
:100BE000A700A500A430A600512000304C204B30B7
:100BF000B700B5010530A700A5001430A6005120AC
:100C00000800272E3C08A0003D08A100A3010030E9
:100C1000EA20031D272E0130BC00BD01BA01BB0133
:100C200000304C204B30B700B5010530A700A500BF
:100C30001430A600512000304C204B30B700B501D5
:100C40000630A700A500A430A60051200800080027
:02400E00EA3096
:00000001FF
